:0200000480007A
:100000006F00C0006F20802C6F20402C93000000F8
:10001000130100009301000013020000930200008E
:100020001303000093030000130400009304000076
:10003000130500009305000013060000930600005E
:100040001307000093070000130800009308000046
:100050001309000093090000130A0000930A00002E
:10006000130B0000930B0000130C0000930C000016
:10007000130D0000930D0000130E0000930E0000FE
:10008000130F0000930F000097020000938202F804
:1000900073905230179100001301C1E4F32240F134
:1000A0009392C2003301510073100134EF20900B82
:1000B000173500001305858B6F20006B8332851088
:1000C000739012148330850003310501833185015B
:1000D000033205028332850203330503833385032C
:1000E000033405048334850483358505033605060A
:1000F00083368506033705078337850703380508E8
:10010000833885080339050983398509033A050AC7
:10011000833A850A033B050B833B850B033C050CA7
:10012000833C850C033D050D833D850D033E050E87
:10013000833E850E033F050F833F850F033505057D
:10014000730020107311011423341100233C31007B
:10015000233041022334510223386102233C7102CF
:1001600023308104233491042338A104233CB104B7
:100170002330C1062334D1062338E106233CF1069F
:10018000233001092334110923382109233C310983
:100190002330410B2334510B2338610B233C710B6B
:1001A0002330810D2334910D2338A10D233CB10D53
:1001B0002330C10F2334D10F2338E10F233CF10F3B
:1001C000F312011423385100F32200102330511090
:1001D000F322101423345110F32230142338511019
:1001E000F3222014233C5110130501006F208033AB
:1010000000000000000000000000000000000000E0
:1010100000000000000000000000000000000000D0
:1010200000000000000000000000000000000000C0
:1010300000000000000000000000000000000000B0
:081040000000000000000000A8
:10200000B367B500B3E7C70093F77700B306C50021
:10201000638407023386C50093070500637ED502FB
:1020200003C705009385150093871700A38FE7FE6C
:10203000E398C5FE67800000E37ED5FE93070500A8
:1020400003B70500938787009385850023BCE7FECF
:10205000E3E8D7FE6780000067800000130101FFFE
:10206000B367C500233081002334110093F7770054
:10207000130405003307C500638207026376E50099
:1020800093F5F50FEFF09FFD8330810013050400F9
:1020900003340100130101016780000093F5F50F7F
:1020A00093968500B3E6B60093970601B3E7D70091
:1020B00093960702B3E6F600E378E5FC9307050084
:1020C0009387870023BCD7FEE3ECE7FE83308100D3
:1020D00013050400033401001301010167800000AF
:1020E00083470500638E07009307050003C71700A9
:1020F00093871700E31C07FE3385A7406780000025
:1021000013050000678000008347050093851500D4
:102110001305150003C7F5FF638A0700E386E7FE92
:102120001B8507003B05E5406780000013050000A4
:102130006FF05FFFB367B50093F77700639E070208
:10214000137886FF330805016378050393070500BC
:102150006F000001938787009385850063F807016E
:1021600083B6070003B70500E386E6FE3385A74084
:102170003306A640138507003386C5006F00400173
:1021800003C705008347F5FF93851500639AE700B1
:1021900013051500E396C5FE1305000067800000D7
:1021A0003B85E740678000009307050003C70500F3
:1021B0009387170093851500A38FE7FEE31807FEAA
:1021C000678000000347050093060002930705009F
:1021D0006318D70003C7170093871700E30CD7FED7
:1021E0009306D0026300D7069306B0026300D704BB
:1021F00083C60700930500006382060413050000F0
:1022000093871700131725001B8606FD83C607005A
:102210003307A700131717003305E600E39206FE05
:10222000638005023305A0406780000083C6170065
:102230009305000093871700E39206FC1305000046
:102240006780000083C6170093051000938717006E
:10225000E39606FA130500006FF09FFE8347050022
:10226000638007049305101017F7FFFF130787D942
:10227000939505030336070013051500B3E6B70071
:10228000630A060097F7FFFF23BE07DA83370700CC
:10229000E39A07FE2330D70083470500E39C07FC41
:1022A0006780000017F7FFFF1307C7D583370700C4
:1022B000638A070097F7FFFF23B607D88337070025
:1022C000E39A07FE2330A7006F000000130101FF0F
:1022D0001305903423341100EFF0DFFC130101FEED
:1022E0001306810093077101130890006F008000AE
:1022F000930707009376F500138706009305000304
:102300006374D800930570053B07B7002380E7008E
:10231000135545001387F7FFE31CF6FC8347810044
:10232000230C0100638207041305101093060600B6
:1023300017F7FFFF130707CD1315050383350700B4
:102340009386160033E6A700638A050097F7FFFF20
:1023500023BA07CE83370700E39A07FE83C7060038
:102360002330C700E39C07FC1301010267800000D3
:10237000130101FF37F8FFFF233411003307050174
:10238000B7E703006378F7141357C5009306076097
:1023900017260000130606C793973600B307F6000A
:1023A00083B70700337505016390070E976500003A
:1023B0009385C5C503B805006302081483378800F8
:1023C0009768000083B808C423B0F500638E170F28
:1023D0008337080093983600B308160193D7C700D7
:1023E0009397A70013E3F70D93E5F70123B0680077
:1023F00073000512971700009387C7C01317470093
:10240000B387E70003B7070063140710033708001A
:10241000B708040023B0E7000337880023B4E700BF
:10242000F3A80810B707E0FFB307F500371800005E
:10243000130705003388070103BF070083BE870029
:1024400003BE070103B387012330E7012334D7011B
:102450002338C701233C670093870702130707024D
:10246000E39C07FD7390081093973600B306F600BF
:1024700023B0B600730005120F10000083308100F6
:10248000130101016780000013F70704630A0702C4
:1024900013F70708631A07041307F00093E7070808
:1024A0006394E50493963600B306D60023B0F60095
:1024B0007300051283308100130101016780000061
:1024C00093E707046FF01FFE9767000023BC07B275
:1024D0006FF01FF0170500001305457CEFF01FD8C3
:1024E00013053000EFF01FDC170500001305857F92
:1024F000EFF0DFD613053000EFF0DFDA171500003C
:102500001305C582EFF09FD513053000EFF09FD97A
:102510001715000013050583EFF05FD41305300095
:10252000EFF05FD883358511130101F82338810658
:10253000233C11062334910623302107233C310527
:10254000233841052334510523306105233C7103B1
:1025500023388103233491032330A103233CB101A9
:102560009307800013040500638AF50E930720008B
:102570006380F506938745FF130710006376F70025
:102580009307F0006392F51A03350411EFF05FDE54
:102590001305040003340107833081078334810667
:1025A0000339010683398105033A0105833A810421
:1025B000033B0104833B8103033C0103833C810211
:1025C000033D0102833D8101130101086FD01FAF5C
:1025D000033785109377370063980706EF0780006D
:1025E000731030000327070083A70700630AF7046E
:1025F0001305101093071004970600009386867841
:1026000017F7FFFF130707A013150503833507000E
:102610009386160033E6A700638A050097F7FFFF4D
:1026200023B207A283370700E39A07FE83C7060099
:102630002330C700E39C07FC13053000EFF09FC672
:1026400013051000EFF01FC6170500001305857D68
:10265000EFF0DFC013053000EFF0DFC403290505FC
:10266000371C0000971400009384C499972B000036
:10267000938B4B99370B0400B70AE0FF976D00006E
:10268000938D4D98176A0000130A4A98B7F9030012
:102690006F0080012334F70023B0FD00B71700005E
:1026A000330CFC00630E3C0B9357CC001394470093
:1026B0003387840003370700E30207FE9387076030
:1026C00093973700B387FB0083BC070093F70C0494
:1026D000638E0706732D0B1037160000B3055C01DF
:1026E00013050C002334B100EFF0DFA4630E0500E6
:1026F00093FC0C088335810063800C0437160000BE
:1027000013050C00EFF0DF8FB387840073100D10FA
:1027100003B70D0023B00700E31E07F623B0FD004A
:102720002330FA006FF09FF71705000013050572BC
:10273000EFF0DFB26FF05FF0170500001305056BD7
:10274000EFF0DFB113053000EFF0DFB51705000043
:1027500013054566EFF09FB013053000EFF09FB40E
:1027600013050900EFF01FB4F32740F1639A07182F
:102770009747000093870789130101ED93D7C7009E
:1027800023308112175800001308C887130405006E
:102790009397A700173500001305C586233411123F
:1027A0009356C5001357C80093E7170097280000F9
:1027B000938848851306F0FF233CF5FE9396A60008
:1027C0001317A700B707002093E61600136717003A
:1027D00093D5C8001313F6039387F70C233CF8FE38
:1027E00023B0D8002330E500B3E7650073900718E5
:1027F00073270018639EE7141356B6009307F00181
:102800009702000093824201F39252307310063B0C
:102810007390073A739052301308F0BF13185801A1
:1028200097E7FFFF93874792B3870701739057108D
:10283000F3270034B387070173900714B7B700007C
:102840009B87071073902730B7E701009B870760CD
:10285000739007307350403017170000130787B983
:102860009307083EB3060701B307F700B70808004F
:1028700017560000233CD67817130000130383F685
:102880009756000023B0F6789388F8039307000169
:102890001308080113D61700B3861701B347F600D3
:1028A000B30507019396C600939757002330D700CE
:1028B0002334B70093F7070213070701B367F60045
:1028C000E31AE3FC13060012930500001305010050
:1028D0009717000023B407F0EFF04FF8B707008018
:1028E0003304F4001305010023348110EFD00FFDF1
:1028F0008330811203340112130101136780000039
:1029000013071000B747290A370608009387F7DE38
:102910001306C6FF1315F7019316E7036F00C001F6
:102920002F20070013D71700B3C7E7009397E703DB
:10293000B3F7D700B3E7E70033F7C70093F5170005
:102940003307A700E39E05FC032007006FF09FFDFF
:102950001705000013058552EFF05F901305300056
:10296000EFF05F9467800000930010001B97000059
:10297000930310009301200063127730930010003E
:102980001B97100093032000930130006318772EEB
:10299000930010001B977000930300089301400000
:1029A000631E772C930010001B97E000B7430000D4
:1029B000930150006314772C930010001B97F001D3
:1029C000B703008093016000631A772A9300F0FF39
:1029D0001B9700009303F0FF930170006310772AA8
:1029E0009300F0FF1B9710009303E0FF930180001A
:1029F000631677289300F0FF1B977000930300F88D
:102A000093019000631C77269300F0FF1B97E00072
:102A1000B7C3FFFF9301A000631277269300F0FF76
:102A20001B97F001B70300809301B000631877246F
:102A3000B72021219B8010121B970000B723212172
:102A40009B8313129301C000631A7722B7202121C0
:102A50009B8010121B971000B74342429B83232494
:102A60009301D000631C7720B72021219B80101296
:102A70001B977000B79390909B8303089301E0002D
:102A8000631E771EB72021219B8010121B97E00048
:102A9000B74348489301F0006312771EB720212105
:102AA0009B8010121B97F001B70300809301000177
:102AB0006316771CB720F1FF9B8050349390C000C1
:102AC000938080671B970000B75334129B83836702
:102AD0009301C0026314771AB720F1FF9B80503432
:102AE0009390C000938080671B974000B763452395
:102AF0009B8303789301D00263127718B7200900F3
:102B00009B8050349390C000938080671B97000097
:102B1000B75334929B8383679301E0026310771667
:102B2000B79009009B8050349390C00093808067D9
:102B30001B974000B76345939B8303789301F00292
:102B4000631E7712930010009B907000930300089F
:102B5000930110016394701213020000930010009F
:102B60001B9770001303070013021200930220004A
:102B7000E31652FE930300089301200163107310C3
:102B800013020000930010001B97E00013000000E8
:102B9000130307001302120093022000E31452FEF5
:102BA000B743000093013001631A730C1302000055
:102BB000930010001B97F0011300000013000000A9
:102BC000130307001302120093022000E31252FEC7
:102BD000B7030080930140016312730A13020000DF
:102BE000930010001B977000130212009302200044
:102BF000E31852FE93030008930150016310770815
:102C00001302000093001000130000001B97E00067
:102C10001302120093022000E31652FEB743000095
:102C200093016001631C77041302000093001000FD
:102C300013000000130000001B97F00113021200A4
:102C400093022000E31452FEB70300809301700149
:102C5000631677029B10F00193030000930180013B
:102C6000639E70009300F0011B90C001930300006D
:102C70009301900163147000631A300013951100E2
:102C800063000500136515007300000013051000B4
:082C900073000000731000C086
:102C9800417373657274696F6E206661696C6564EF
:102CA8003A2061646472203E3D202831554C203C16
:102CB8003C203132292026262061646472203C2081
:102CC8003633202A202831554C203C3C20313229EB
:102CD8000A00000000000000417373657274696F98
:102CE8006E206661696C65643A20212870745B33D4
:102CF8005D5B616464722F2831554C203C3C203167
:102D080032295D20262030783038302920262620A8
:102D18006361757365203D3D203078660A000000C8
:102D2800417373657274696F6E206661696C65645E
:102D38003A206E6F64650A00417373657274696F37
:102D48006E206661696C65643A20757365725F6DA3
:102D5800617070696E675B616464722F2831554CCD
:102D6800203C3C203132295D2E61646472203D3D57
:102D780020300A0000000000417373657274696FA7
:102D88006E206661696C65643A202122696C6C6505
:102D980067616C20696E737472756374696F6E22F3
:102DA8000A00000000000000417373657274696FC7
:102DB8006E206661696C65643A2070745B335D5B94
:102DC800616464722F2831554C203C3C20313229F3
:102DD8005D20262030783034300A000000000000E2
:102DE800417373657274696F6E206661696C65649E
:102DF8003A2070745B335D5B616464722F283155CF
:102E08004C203C3C203132295D2026203078303857
:102E1800300A000000000000417373657274696F26
:102E28006E206661696C65643A2074662D3E657033
:102E38006320252034203D3D20300A00000000009A
:102E4800417373657274696F6E206661696C65643D
:102E58003A202122756E6578706563746564206513
:102E68007863657074696F6E220A000000000000C4
:102E7800417373657274696F6E206661696C65640D
:102E88003A202122756E737570706F7274656420B4
:0C2E980073617470206D6F6465220A0085
:040000058000000077
:00000001FF
